:100000000C94280018950000189500001895000021
:10001000189500001895000018950000189500002C
:10002000189500001895000018950000189500001C
:10003000189500001895000018950000189500000C
:1000400018950000189500001895000018950000FC
:100050008FE181BD87E181BD8FE58DBFC0E4E8E31D
:100060004E2E88E08EBFD8E0F8E05F2EEEEFF7E08E
:10007000A0E6B0E088278D933197E9F70E94BE0A89
:1000800066248CE00E94100BA198A098D39ADB9A6A
:10009000A09AA19AA99880E08093620080E0809362
:1000A000610080E0809360008AE695E0A8E6B0E019
:1000B0008D939C9381E08093660081E0809367003C
:1000C00081E080936A0081E080936B0070916C0006
:1000D0007F7770936C0070916C007F7B70936C00E5
:1000E00070916C007F7D70936C0070916C007D7FCF
:1000F00070936C0070916D007F7770936D007091BC
:100100006D00706470936D0070916C0070617093FD
:100110006C0070916C00746070936C0070916C0056
:10012000786070936C0080E080936E000E94A60A55
:100130000E94A20A0E943A0B002F0F3081E009F0C2
:1001400080E08F930027ACE6B0E08C9186FB0EF444
:1001500001E040E0041781E009F080E09F918923ED
:10016000882311F40C94C100ACE6B0E08C9187FBBD
:10017000882780F9809580FBACE6B0E08C9187F908
:100180008C930E943A0B002F0B3081E009F080E045
:100190008F930027ACE6B0E08C9187FB0EF401E072
:1001A00040E0041781E009F080E09F9189238823D3
:1001B00011F40C94EB00ACE6B0E08C9186FB882740
:1001C00080F9809580FBACE6B0E08C9186F98C9349
:1001D00080E080936E000E943A0B002F0C3081E08B
:1001E00009F080E08F930027ACE6B0E08C9186FBAD
:1001F0000EF401E040E0041781E009F080E09F91F7
:1002000089238F930027ACE6B0E08C9187FB0EF436
:1002100001E040E0041781E009F080E09F9189232C
:10022000882311F40C942101ACE6B0E08C9181FBA1
:10023000882780F9809580FBACE6B0E08C9181F94D
:100240008C930E943A0B002F073011F00C94370169
:1002500070916C007F7770936C0070916C007F7B65
:1002600070936C0070916C007D7F70936C000E94A5
:100270003A0B002F003081E009F080E08F930027D7
:10028000ACE6B0E08C9187FB0EF401E041E004178E
:1002900081E009F080E09F9189238F930027ACE6ED
:1002A000B0E08C9186FB0EF401E040E0041781E0A1
:1002B00009F080E09F9189238F930027ACE6B0E09E
:1002C0008C9181FB0EF401E040E0041781E009F01D
:1002D00080E09F918923882311F40C9471010E947E
:1002E00077090E943A0B002F013081E009F080E08D
:1002F0008F930027ACE6B0E08C9187FB0EF401E011
:1003000041E0041781E009F080E09F9189238F93F9
:100310000027ACE6B0E08C9186FB0EF401E040E0F3
:10032000041781E009F080E09F9189238F930027D3
:10033000ACE6B0E08C9181FB0EF401E040E00417E4
:1003400081E009F080E09F918923882311F40C94C7
:10035000AB010E9489090E943A0B002F023081E014
:1003600009F080E08F930027ACE6B0E08C9187FB2A
:100370000EF401E041E0041781E009F080E09F9174
:1003800089238F930027ACE6B0E08C9186FB0EF4B6
:1003900001E040E0041781E009F080E09F918923AB
:1003A0008F930027ACE6B0E08C9181FB0EF401E066
:1003B00040E0041781E009F080E09F9189238823C1
:1003C00011F40C94E5010E949B090E943A0B002F46
:1003D000033081E009F080E08F930027ACE6B0E0C5
:1003E0008C9187FB0EF401E041E0041781E009F0F5
:1003F00080E09F9189238F930027ACE6B0E08C9139
:1004000086FB0EF401E040E0041781E009F080E093
:100410009F9189238F930027ACE6B0E08C9181FBFC
:100420000EF401E040E0041781E009F080E09F91C4
:100430008923882311F40C941F020E94F0090E9462
:100440003A0B002F003081E009F080E08F93002705
:10045000ACE6B0E08C9187FB0EF401E040E00417BD
:1004600081E009F080E09F9189238F930027ACE61B
:10047000B0E08C9186FB0EF401E040E0041781E0CF
:1004800009F080E09F9189238F930027ACE6B0E0CC
:100490008C9181FB0EF401E040E0041781E009F04B
:1004A00080E09F918923882311F40C946402ACE6C8
:1004B000B0E08C9184FB882780F9809580FBACE6C6
:1004C000B0E08C9184F98C930E943A0B002F01309C
:1004D00081E009F080E08F930027ACE6B0E08C91DA
:1004E00087FB0EF401E040E0041781E009F080E0B2
:1004F0009F9189238F930027ACE6B0E08C9186FB17
:100500000EF401E040E0041781E009F080E09F91E3
:1005100089238F930027ACE6B0E08C9181FB0EF429
:1005200001E040E0041781E009F080E09F91892319
:10053000882311F40C94A902ACE6B0E08C9183FB03
:10054000882780F9809580FBACE6B0E08C9183F938
:100550008C930E943A0B002F023081E009F080E07A
:100560008F930027ACE6B0E08C9187FB0EF401E09E
:1005700040E0041781E009F080E09F9189238F9388
:100580000027ACE6B0E08C9186FB0EF401E040E081
:10059000041781E009F080E09F9189238F93002761
:1005A000ACE6B0E08C9181FB0EF401E040E0041772
:1005B00081E009F080E09F918923882311F40C9455
:1005C000EE02ACE6B0E08C9182FB882780F9809542
:1005D00080FBACE6B0E08C9182F98C930E943A0BE0
:1005E000002F033081E009F080E08F930027ACE614
:1005F000B0E08C9187FB0EF401E040E0041781E04D
:1006000009F080E09F9189238F930027ACE6B0E04A
:100610008C9186FB0EF401E040E0041781E009F0C4
:1006200080E09F9189238F930027ACE6B0E08C9106
:1006300081FB0EF401E040E0041781E009F080E066
:100640009F918923882311F40C943303BB27ABE3D8
:100650008C9183FB882780F9809580FBBB27ABE3D7
:100660008C9183F98C930E943A0B002F003081E02B
:1006700009F080E08F930027ACE6B0E08C9181FB1D
:100680000EF401E041E0041781E009F080E09F9161
:1006900089238F930027ACE6B0E08C9187FB0EF4A2
:1006A00001E040E0041781E009F080E09F91892398
:1006B000882311F40C946E03ACE6B0E08C9180FBBF
:1006C000882780F9809580FBACE6B0E08C9180F9BA
:1006D0008C9370916D007F7770936D000E943A0B40
:1006E000002F003081E009F080E08F930027ACE616
:1006F000B0E08C9181FB0EF401E041E0041781E051
:1007000009F080E09F9189238F930027ACE6B0E049
:100710008C9187FB0EF401E041E0041781E009F0C1
:1007200080E09F918923882311F40C9499030E94FF
:10073000020A0E943A0B002F013081E009F080E0AC
:100740008F930027ACE6B0E08C9181FB0EF401E0C2
:1007500041E0041781E009F080E09F9189238F93A5
:100760000027ACE6B0E08C9187FB0EF401E041E09D
:10077000041781E009F080E09F918923882311F418
:100780000C94C4030E94140A0E943A0B002F0230FA
:1007900081E009F080E08F930027ACE6B0E08C9117
:1007A00081FB0EF401E041E0041781E009F080E0F4
:1007B0009F9189238F930027ACE6B0E08C9187FB53
:1007C0000EF401E041E0041781E009F080E09F9120
:1007D0008923882311F40C94EF030E94260A0E94B7
:1007E0003A0B002F033081E009F080E08F9300275F
:1007F000ACE6B0E08C9181FB0EF401E041E004171F
:1008000081E009F080E09F9189238F930027ACE677
:10081000B0E08C9187FB0EF401E041E0041781E029
:1008200009F080E09F918923882311F40C941A0425
:100830000E947B0A0E94A60A0027ACE6B0E08C91D9
:1008400086FB0EF401E040E0041781E009F080E04F
:100850008F930027ACE6B0E08C9184FB0EF401E0AE
:1008600040E0041781E009F080E09F9189238F9395
:100870000027ACE6B0E08C9183FB0EF401E041E090
:10088000041781E009F080E09F9189238F9300276E
:10089000ACE6B0E08C9181FB0EF401E040E004177F
:1008A00081E009F080E09F918923882311F40C9462
:1008B0007D04E6EBF7E10E949B0AA8E2B8E0E2E6DD
:1008C000F0E00E94910B0E94930AE8EBF7E10E948E
:1008D0009B0AA8E2B8E0E1E6F0E00E94910B0E94DA
:1008E000930AE8EBF7E10E949B0AA8E2B8E0E0E691
:1008F000F0E00E94910B0E94930A0027ACE6B0E062
:100900008C9186FB0EF401E040E0041781E009F0D1
:1009100080E08F930027ACE6B0E08C9184FB0EF46E
:1009200001E041E0041781E009F080E09F91892314
:100930008F930027ACE6B0E08C9183FB0EF401E0CE
:1009400041E0041781E009F080E09F9189238F93B3
:100950000027ACE6B0E08C9181FB0EF401E040E0B2
:10096000041781E009F080E09F918923882311F426
:100970000C94DE04EAEBF7E10E949B0AA8E2B8E0DF
:10098000E2E6F0E00E94910B0E94930AE8EBF7E1A7
:100990000E949B0AA8E2B8E0E1E6F0E00E94910B19
:1009A0000E94930AE8EBF7E10E949B0AA8E2B8E0F4
:1009B000E0E6F0E00E94910B0E94930A8FEB11E0B9
:1009C0000E94B50A0027ACE6B0E08C9186FB0EF4DD
:1009D00001E040E0041781E009F080E08F930027F8
:1009E000ACE6B0E08C9184FB0EF401E040E004172B
:1009F00081E009F080E09F9189238F930027ACE686
:100A0000B0E08C9182FB0EF401E041E0041781E03C
:100A100009F080E09F9189238F930027ACE6B0E036
:100A20008C9181FB0EF401E040E0041781E009F0B5
:100A300080E09F918923882311F40C944305E6EB11
:100A4000F7E10E949B0AA8E2B8E0E8E6F0E00E9425
:100A50008A0B0E94930AE2ECF7E10E949B0AA8E24B
:100A6000B8E0E6E6F0E00E94910B0E94930AE2EC07
:100A7000F7E10E949B0AA8E2B8E0E7E6F0E00E94F6
:100A8000910B0E94930A0027ACE6B0E08C9186FBA4
:100A90000EF401E040E0041781E009F080E08F935C
:100AA0000027ACE6B0E08C9184FB0EF401E041E05D
:100AB000041781E009F080E09F9189238F9300273C
:100AC000ACE6B0E08C9182FB0EF401E041E004174B
:100AD00081E009F080E09F9189238F930027ACE6A5
:100AE000B0E08C9181FB0EF401E040E0041781E05E
:100AF00009F080E09F918923882311F40C94A405C8
:100B0000E4ECF7E10E949B0AA8E2B8E0E8E6F0E036
:100B10000E948A0B0E94930AE2ECF7E10E949B0A72
:100B2000A8E2B8E0E6E6F0E00E94910B0E94930A8A
:100B3000E2ECF7E10E949B0AA8E2B8E0E7E6F0E009
:100B40000E94910B0E94930A8FE711E00E94B50A60
:100B50000027ACE6B0E08C9186FB0EF401E040E0AB
:100B6000041781E009F080E08F930027ACE6B0E045
:100B70008C9181FB0EF401E041E0041781E009F063
:100B800080E09F918923882311F40C94EB05ECEC11
:100B9000F7E10E949B0AA8E2B8E0E5E6F0E00E94D7
:100BA000910B0E94930AE8EBF7E10E949B0AA8E2EE
:100BB000B8E0E4E6F0E00E94910B0E94930AE8EBB3
:100BC000F7E10E949B0AA8E2B8E0E3E6F0E00E94A9
:100BD000910B0E94930A8FEB11E00E94B50A002747
:100BE000ACE6B0E08C9186FB0EF401E040E0041727
:100BF00081E009F080E08F930027ACE6B0E08C91B3
:100C000081FB0EF401E041E0041781E009F080E08F
:100C10009F918923882311F40C943206E0EDF7E1CB
:100C20000E949B0AA8E2B8E0E8E6F0E00E948A0B86
:100C30000E94930AE2ECF7E10E949B0AA8E2B8E066
:100C4000EAE6F0E00E94910B0E94930AE2ECF7E1E1
:100C50000E949B0AA8E2B8E0EBE6F0E00E94910B4C
:100C60000E94930A8FEB10E10E94B50A0027ACE6C0
:100C7000B0E08C9186FB0EF401E040E0041781E0C7
:100C800009F080E08F930027ACE6B0E08C9181FB07
:100C90000EF401E041E0041781E009F080E09F914B
:100CA0008923882311F40C945906E4EDF7E10E949E
:100CB0009B0A0027ACE6B0E08C9187FB0EF401E0C4
:100CC00041E0041711F00C946D068FE71FE00E94BD
:100CD000B50AE6EDF7E10E949B0A0027ACE6B0E01A
:100CE0008C9187FB0EF401E040E0041781E009F0ED
:100CF00080E08F930027ACE6B0E08C9180FB0EF48F
:100D000001E041E0041781E009F080E09F91892330
:100D10008F930027ACE6B0E08C9186FB0EF401E0E7
:100D200040E0041781E009F080E09F9189238F93D0
:100D30000027BB27A5E38C9180FB0EF401E041E086
:100D4000041781E009F080E09F918923882311F442
:100D50000C94B706ADE6B0E08C9186FB882780F94D
:100D6000809580FBADE6B0E08C9186F98C930027EE
:100D7000ACE6B0E08C9187FB0EF401E040E0041794
:100D800081E009F080E08F930027ACE6B0E08C9121
:100D900080FB0EF401E041E0041781E009F080E0FF
:100DA0009F9189238F930027ACE6B0E08C9186FB5E
:100DB0000EF401E040E0041781E009F080E09F912B
:100DC00089238F930027ADE6B0E08C9186FB0EF46B
:100DD00001E041E0041781E009F080E09F91892360
:100DE000882311F40C94FC068FE71FE00E94B50ADB
:100DF000EAEDF7E10E949B0A0027ACE6B0E08C9197
:100E000086FB0EF401E041E0041781E009F080E088
:100E10008F930027ACE6B0E08C9187FB0EF401E0E5
:100E200040E0041781E009F080E09F9189238F93CF
:100E300000916E00003081E009F080E09F918923ED
:100E4000882311F40C9436070E94A60A8FE715E058
:100E50000E94B50AEEEDF7E10E949B0A8FEB13E0CA
:100E60000E94B50AE8EEF7E10E949B0A0027ACE673
:100E7000B0E08C9186FB0EF401E041E0041781E0C4
:100E800009F080E08F930027ACE6B0E08C9187FBFF
:100E90000EF401E040E0041781E009F080E09F914A
:100EA00089238F9300916E00013081E009F080E08A
:100EB0009F918923882311F40C9470070E94A60A3D
:100EC0008FE714E00E94B50AE6EFF7E10E949B0A63
:100ED0008FEB15E00E94B50AE2E0F8E10E949B0A60
:100EE0000027ACE6B0E08C9186FB0EF401E041E017
:100EF000041781E009F080E08F930027ACE6B0E0B2
:100F00008C9187FB0EF401E040E0041781E009F0CA
:100F100080E09F9189238F9300916E00023081E0E1
:100F200009F080E09F918923882311F40C94AA078B
:100F30000E94A60A8FE715E00E94B50AECE0F8E1EE
:100F40000E949B0A8FEB14E00E94B50AE4E1F8E1ED
:100F50000E949B0A0027ACE6B0E08C9186FB0EF461
:100F600001E041E0041781E009F080E08F93002761
:100F7000ACE6B0E08C9187FB0EF401E040E0041792
:100F800081E009F080E09F9189238F9300916E00AA
:100F9000033081E009F080E09F918923882311F4D8
:100FA0000C94E4070E94A60A8FE714E00E94B50A99
:100FB000EEE1F8E10E949B0A8FEB11E00E94B50A76
:100FC000EAE2F8E10E949B0A0027ACE6B0E08C91CF
:100FD00086FB0EF401E041E0041781E009F080E0B7
:100FE0008F930027ACE6B0E08C9187FB0EF401E014
:100FF00040E0041781E009F080E09F9189238F93FE
:1010000000916E00043081E009F080E09F91892317
:10101000882311F40C941E080E94A60A8FE715E09D
:101020000E94B50AEAE3F8E10E949B0A8FEB11E007
:101030000E94B50AE2E4F8E10E949B0A8EEA93E07E
:101040000E94610BA0E6B0E08C918F5F8C930091C1
:1010500060000B3318F011F00C9430080C94380831
:1010600080E080936000A1E6B0E08C918F5F8C936C
:10107000009161000B3318F011F00C9441080C94AE
:10108000490880E080936100A2E6B0E08C918F5F18
:101090008C9300916200073118F011F00C94520803
:1010A0000C945A0880E080936200A7E6B0E08C912F
:1010B0008F5F8C9300916600073081E008F080E03C
:1010C0008F93009167000F3180E010F009F081E00C
:1010D0009F918923882311F40C947608A6E6B0E04A
:1010E0008C918F5F8C9381E0809367000091660004
:1010F000073080E010F009F081E08F9300916600E6
:101100000C3081E008F080E09F9189238F9300915B
:1011100067000E3180E010F009F081E09F91892393
:10112000882311F40C949C08A6E6B0E08C918F5FA4
:101130008C9381E080936700009166000C3081E021
:1011400009F080E08F93009167000D3180E010F08E
:1011500009F081E09F918923882311F40C94BA0847
:1011600081E08093660081E080936700A8E6B0E0AC
:101170000E948D0A0027ACE6B0E08C9186FB0EF44D
:1011800001E041E0041781E009F080E08F9300273F
:10119000ACE6B0E08C9185FB0EF401E041E0041771
:1011A00081E009F080E09F918923882311F40C9459
:1011B000DE08AEE6B0E08C918F5F8C9300916E00FC
:1011C000053011F00C94E70880E080936E00ACE6E7
:1011D000B0E08C9185FB882780F9809580FBACE698
:1011E000B0E08C9185F98C9340916A000091660083
:1011F000041781E009F080E08F9340916B0000912B
:101200006700041781E009F080E09F9189238F93A4
:101210004091650000916200041781E009F080E0D0
:101220009F9189238F93409164000091610004177E
:1012300081E009F080E09F9189238F930027ACE63D
:10124000B0E08C9180FB0EF401E041E0041781E0F6
:1012500009F080E09F918923882311F40C943809C8
:10126000A89A70916D00706870936D000C943E099F
:10127000A89870916D00706470936D000027ADE6C2
:10128000B0E08C9187FB0EF401E041E0041781E0AF
:1012900009F080E08F930027ACE6B0E08C9180FBF2
:1012A0000EF401E041E0041781E009F080E09F9135
:1012B00089238F930027BB27A5E38C9180FB0EF435
:1012C00001E040E0041781E009F080E09F9189236C
:1012D000882311F40C94710970916C007E7F7093D7
:1012E0006C000C9496000C949A00F894FFCFA1E641
:1012F000B0E08C918F5F8C93009161000B3318F0FC
:1013000011F00C9485090C94880980E080936100A9
:101310000895A2E6B0E08C918F5F8C9300916200FB
:10132000073118F011F00C9497090C949A0980E099
:10133000809362000895A7E6B0E08C918F5F8C9354
:1013400000916600073081E008F080E08F93009103
:1013500067000F3180E010F009F081E09F91892350
:10136000882311F40C94B70981E080936700009101
:101370006600073080E010F009F081E08F93009163
:1013800066000C3081E008F080E09F9189238F9304
:10139000009167000E3180E010F009F081E09F912C
:1013A0008923882311F40C94D80981E08093670085
:1013B000009166000C3081E009F080E08F9300918D
:1013C00067000D3180E010F009F081E09F918923E2
:1013D000882311F40C94EF0981E08093670008954D
:1013E000A6E6B0E08C918F5F8C93009166000C3084
:1013F00018F011F00C94FE090C94010A81E080931E
:1014000066000895A4E6B0E08C918F5F8C93009104
:1014100064000B3318F011F00C94100A0C94130AAA
:1014200080E0809364000895A5E6B0E08C918F5F22
:101430008C9300916500073118F011F00C94220A8A
:101440000C94250A80E0809365000895ABE6B0E037
:101450008C918F5F8C9300916A00073081E008F0D7
:1014600080E08F9300916B000F3180E010F009F065
:1014700081E09F918923882311F40C94420A81E032
:1014800080936B0000916A00073080E010F009F053
:1014900081E08F9300916A000C3081E008F080E0D9
:1014A0009F9189238F9300916B000E3180E010F0A3
:1014B00009F081E09F918923882311F40C94630A39
:1014C00081E080936B0000916A000C3081E009F0AC
:1014D00080E08F9300916B000D3180E010F009F0F7
:1014E00081E09F918923882311F40C947A0A81E08A
:1014F00080936B000895AAE6B0E08C918F5F8C9387
:1015000000916A000C3018F011F00C94890A0C94C8
:101510008C0A81E080936A000895ED91FC913196E8
:10152000FC93EE930895A8E2B8E08D91882311F022
:1015300071D0FBCF08950E94700B802D11F06AD0FE
:10154000FACF089582E06CD016D012C081E068D046
:1015500012D080E865C08FE7213039F08FEB223060
:1015600021F08FE8233009F08FEC810F0C94100BE1
:1015700080E856D0089583E09927A3C08AEF90E0D1
:101580000E94610BD79AD69AD59AD49AD29AD09AB9
:10159000D898EF93FF93E1E1F1E00E94310BFF91C6
:1015A000EF91DA98DF98DE98DD9ADC9ADA9AEF9379
:1015B000FF93E1E1F1E00E94310BFF91EF91DA98A6
:1015C0007DD0DA9AEF93FF93E1E1F1E00E94310BD5
:1015D000FF91EF91DA9872D0DA9AEF93FF93E1E1FD
:1015E000F1E00E94310BFF91EF91DA9867D0DC981F
:1015F000DA9AEF93FF93E1E1F1E00E94310BFF9162
:10160000EF91DA985BD088E20BD08EE009D086E0CB
:1016100007D00895D89A829505D004D04FD0089568
:10162000D898F9CF859510F4DC9A01C0DC9885959F
:1016300010F4DD9A01C0DD98859510F4DE9A01C0A2
:10164000DE98859510F4DF9A01C0DF98DA9AEF935F
:10165000FF93E1E1F1E00E94310BFF91EF91DA9805
:1016600008953197F1F70895689462F80895E89421
:1016700062F8089500E18FEF82BB8FE081BB80EFBD
:1016800082BB84E18A95F1F7849B00E0859B04E0AE
:10169000869B08E0879B0CE080EF81BB8FE082BBDC
:1016A00084E18A95F1F78827809B80E0819B81E027
:1016B000829B82E0839B83E0080F089581E090E0A5
:1016C00000C0EF93FF93EE27E82BE92B31F0EDEC10
:1016D000FAE03197F1F70197D1F7FF91EF91089573
:1016E000C895319600200895000F111F221F331F47
:1016F000089500951095209530950F5F1F4F2F4F3F
:101700003F4F0895019110810EC0019111912191D7
:1017100030810BC00191108117FF05C03FEF2FEF03
:1017200004C0008111272227332737FF03C0E1DFE0
:101730008DE28D93CF93DF93CF92DF92EF92AA2425
:10174000BB24CC24DD24EE2440E2CAE0DD2755E0B2
:1017500093E38881890F87FD9F7083FD907F891BAC
:1017600089935A95A9F7C0DFAA1CBB1CCC1CDD1CB1
:10177000EE1C4A9551F7E894EFE0FF2782910ED0D6
:10178000EB30E0F71EF068948A2D0CD088278D93FB
:10179000EF90DF90CF90DF91CF910895982F8295B1
:1017A00001D0892F8F70805D26F0803309F4089571
:1017B00068948D93089500003A0054696D653A204D
:1017C00000002F00446174653A200000543A200064
:1017D000443A20005400534D000054310000446549
:1017E0007369676E657200005261736F6F6C20538E
:1017F00068697269000053747564656E74204944A9
:1018000000003834383137373433000054656163B1
:10181000686572004D722E52617A61766900556E6C
:1018200065766572736974790000617A6164206B12
:1018300065726D616E73686168004C65637475658F
:101840007200417263686974656374756572204CD7
:0418500061620000D1
:00000001FF
